S10601007E01A1D8
S12301200205060001030700020408000305090001040A00010B0C00020C0D00030D0E0024
S1230140040E0F00050B0F00060A1100060712000708130008091400090A10000F1114007D
S12301600B1012000C1113000D1214000E1013000101020203030404050506060707080872
S123018009090A0A0B0B0C0C0D0D0E0E0F0F10101111121213131414212114050A05050888
S12301A0217E0A820D0A00040D0A0A0043555252454E5420524F4F4D2049533A040D0A0043
S12301C00054554E4E454C53204C45414420544F3A040D0A0A004D4F5645204F52205348E7
S12301E04F4F543F20042057484552453F20040D0A00004920484541522057494E4753045C
S12302000D0A000049204645454C2041204452414654040D0A00004920534D454C4C2041EA
S12302202057554D50555321040D0A0000594F5520484156452052554E204F5554204F464A
S123024020535550504C49455320414E442057494C4C20535441525645040D0A00005959F8
S123026059494949494545454545452E2E2E2E20594F552046454C4C20494E544F2041206C
S1230280504954040D0A0000414152525252474747474848482E2E2E2E20594F5520484116
S12302A056452053484F5420594F555253454C46040D0A0000432048204F204D2050202056
S12302C04352554E4348204D554E43482047554C50210D0A00005448452057554D5055533A
S12302E020474F5420594F5521040D0A0000594F55204C4F4F5345202848454520484545EC
S123030029040D0A000042204F204E204B202120040D0A0000474F4F4420464F5220594F97
S12303205521202D20594F5520474F542048494D042057495448204120524F434B21040D8F
S12303400A0000535550504C4945532057494C4C204C41535420042044415953040D0A00DE
S123036000424154204D4947524154494F4E202D204849444520414E4420574149540D0AF2
S1230380000020204F4E4520434F4C4F4E59204F46204241545320484153204D4F564544AD
S12303A0040D0A00004E49434520474F494E472C20594F552053484F5420594F55525345BD
S12303C04C460D0A00002020414E4420484156452055534544204D45444943414C205355F1
S12303E050504C494553040D0A000057484F4F4F50532120424154532052454C4F4341544D
S12304004520594F550D0A00002020594F55204C4F535420534F4D4520535550504C49452A
S123042053040D0A0000544855442120594F55204F4E4C592044415A45442048494D040DDE
S12304400A00004D4953534544040D0A00004C4F4F4B2C20594F5520464F554E442004412F
S1230460205448524F57494E4720524F434B04535550504C4945530D0A0000202046524FE0
S12304804D20414E4F544845522028454154454E292048554E544552040D0A000052415404
S12304A053204541542048414C4620594F555220535550504C494553040D0A0000524F43AD
S12304C04B20534C4944452120412054554E4E454C20495320434C4F5345440457415443FB
S12304E0482049542104202D205448452057554D505553204953204157414B45040D0A000F
S12305000057494C442053484F54202D20040D0A0000424947204445414C2C20594F552050
S123052053484F54204120424154040D0A00004120444F574E44524146542048415320538D
S123054055434B454420544845204152524F5720494E544F204120504954040D0A00005943
S12305604F55204A5553542053544550504544204F4E2048495320464C4950504552210420
S12305800D0A0A00444F20594F552057414E5420544F20504C415920414741494E3F200430
S12305A00D0A0000444F20594F552057414E5420544F2053454520412043415645204D4108
S12305C0503F20040D0A000057454C434F4D4520544F205448452057554D505553204341C8
S12305E05645532C0D0A0000444F20594F55205749534820494E535452554354494F4E53E6
S12306003F20040A20574841543F20040D0A00005448414E4B20594F552C2043414D452086
S1230620414741494E20534F4D4554494D452E040D0A000053484F4F5420574841543F0D5D
S12306400A0000594F552048415645204E4F204152524F5753204F5220524F434B53042009
S12306602D20594F552043414E2754204745542054484552452046524F4D2048455245048B
S12306800D0A0A00524F4F4D2020202054554E4E454C532020202020204954454D0A040D45
S12306A00A00005448495320434156452048415320323020494E544552434F4E4E4543548B
S12306C0454420524F4F4D530D0A00005448452057554D5055532049532041534C4545503E
S12306E020494E204F4E4520414E44204D555354204245204B494C4C45440D0A00004946BF
S123070020484520283F292046494E445320594F552048452057494C4C2045415420594F00
S1230720550D0A0000494620594F552057414B452048494D205550204845204D4159204D71
S12307404F56450D0A00004C4F4F4B204F555420464F52204241545320414E4420504954F6
S1230760530D0A00005741524E494E47532041524520464F522048415A4152445320312005
S1230780524F4F4D20415741590D0A0000594F5520484156452035204152524F57532041BA
S12307A04E442041204C494D495445442053544F5245204F4620535550504C4945530D0A0C
S12307C00000454143482053484F54204D415920474F205448524F554748203120544F2074
S12307E03320434F4E4E454354454420524F4F4D530D0A0000594F55204D4159204D414B4B
S1230800452031204D4F5645204F522053484F542045414348204441590D0A00005748459E
S12308204E20594F5520415245204F5554204F46204152524F5753204C4F4F4B20464F522A
S123084020524F434B530D0A0000202057484943482043414E204245205448524F574E206D
S1230860494E544F204F4E4C59203120524F4F4D0D0A00002020414E44204D4159204B4945
S12308804C4C205448452057554D5055530D0A0000202020202020202020474F4F44204CDE
S12308A055434B0D0A0A04FF0114300909AE02AF00BE0114AF0235EE0239300909AE04AFF2
S12308C000AE02AF043531313131EE0039BD08A7C603F7010B7F0112BD102481202609F610
S12308E0010BC10327F22028810D2724812C272081302D3A813922367A010B2731840F3625
S1230900B60112164848481B1B331BB7011220C8B7010EB601122712CE0170A10127090805
S1230920088C019826F52006A600BD08BA39CE01A4BD102ACE01E6BD102A20944D2A0ABDDF
S12309401030BD1030BD103039BD08A7BD1030CE01704A270508084A26FBA6018109220331
S1230960BD1030BD0983BD08BA39BD08A7CE033FBD102AB6010DBD0983CE0357BD102ABD19
S123098008BA397F010B7C010B800A2AF98B0A7A010B36B6010B27058A30BD1027328A30BF
S12309A0BD10273937B601190C490C49BB0118F601190C59490C59490CFB0119B901180C16
S12309C0CB198B36B70118F701193339B701108632B7010BFF0114FE01147A010BBD09A4C7
S12309E0815523060881AA2301087D010B2710A6002BE4BD0A166D0327085D26DA2003B66E
S1230A000110FE011439BD09A4841F811422F74D27F4BD0A1639364A48484CCE01204A2780
S1230A20030820FA3239364A484CCE01704A27030820FA3239BD102436810D2707BD1024FA
S1230A40810D26F93239BD09A4847F816422F7A10023034F200286010839BD0A16E100272A
S1230A600AE1012706E10227025F39C60139CE0311BD102A7C010F39CE02EABD102A7C01E9
S1230A800F39CE05C4BD102ABD0A3584DF8159270C814E270ECE0603BD102A20E5CE069FC6
S1230AA0BD102ABD0AF1BD0BAACE05A0BD102ABD0A3584DF8159270C814E270BCE0603BDA6
S1230AC0102A20E5BD0EF1CE0580BD102ABD0A3584DF815927CD814E2708CE0603BD102AD4
S1230AE020E5CE060CBD102ACE01A4BD102A7E1038BD0B698601B7010BC657F7011CBD0B72
S1230B008EC650F7011CBD09A484014CB7010BBD0B8EC642F7011CBD09A484034CB7010BA9
S1230B20BD0B8EBD0A066D0326F9B7010CCE01706D01261DC61437BD0A06BD0A266D0127EB
S1230B400A8B07811423F3801420EF33E7015A26E57F010ABD0A06478B0AB7010D8605B7ED
S1230B6001167F01117F010F39CE012086036D002A026300084A26F66F00088C017026EC99
S1230B8001CE01706F0108088C019826F739F6010B37BD0A066D0326F9F6011CE703C1576C
S1230BA02603B7011F335A26E8397A010D7D010A2303BD0BF2BD0C137D010F230139CE01D8
S1230BC0D2BD102ABD0A3584DF8153270C814D270DCE0603BD102A20E5BD0D292003BD0E2C
S1230BE0CC7D010F230139CE01A4BD102ABD0F3E20B8CE019ABD0A464D2617B6011FBD0A52
S1230C0016C601BD09CCB7011F6F03BD0A16C657A703397D010D2A0ACE0229BD102ABD0AC5
S1230C207839B6010CBD0A16E603C1422605BD0CC820E0C1572609BD0CEF7D010F230139CE
S1230C40C1502604BD0CE539A600BD0C9BA601BD0C9BA602BD0C9BCE01A8BD102AB6010C1C
S1230C60BD093CCE01BDBD102AB6010CBD0A16BD09A48407B7010BA602E601E702E600E74E
S1230C8001A7007A010B26EFA600BD093CA601BD093CA602BD093CBD096A39BD08A74D2BC5
S1230CA023BD0A16A60381502606CE0200BD102A81422606CE01EFBD102A81572606CE024B
S1230CC013BD102ABD08BA39BD08A7CE03E7BD102ABD0A06B7010CF6010D17575710B70111
S1230CE00DBD08BA39CE025ABD102ABD0A7839BD08A77D010A2225CE01A4BD102ACE04DC3F
S1230D00BD102ACE055BBD102ACE01A4BD102ACE04E6BD102A7C010ABD08BA39CE02B1BD1D
S1230D20102ABD0A78BD08BA397D01162604BD0E07397F011E7F01177A0116CE01A4BD10AF
S1230D402ACE01E6BD102ACE0103FF0108B6010CB7011DC601F70113BD08CD4D2721A700A7
S1230D60087C0113B6010E810D2714F60113C10426E3BD08CD4D2707B6010E810D26F37D7B
S1230D80010A2215CE01A4BD102ACE04DCBD102ACE04E6BD102A7C010A7A01132601397D5D
S1230DA0011E2222FE01087C0109E60037B6011DBD0A5A5D2217CE04FDBD102ACE04DCBD66
S1230DC0102A7C011E31B6011DBD09CC3632B7011DBD0A16A60381572607BD0A6E7C010F1A
S1230DE03981422609BD0E757D011723013981502609BD0E887D0117230139B6011DB101C7
S1230E000C2696BD0E9B397D01112607CE0630BD102A397A0111CE01E6BD102ABD08CDCEDF
S1230E2001A4BD102A4D27EEF6010CBD0A5A5D220DCE043FBD102ACE065FBD102A39BD0ACE
S1230E4016E603C157270EC1422603BD0F6FCE043FBD102A39CE01A0BD0A464D2310CE03CD
S1230E6002BD102ABD0A6ECE0331BD102A39CE0422BD102A39CE0198BD0A464D23097C0180
S1230E8017CE050EBD102A39CE0199BD0A464D23097C0117CE052BBD102A39CE019ABD0A46
S1230EA0464D231ECE03A1BD102AB6010D810522087C010D74010D20058605B7010DBD0936
S1230EC06A39CE0284BD102ABD0A7839CE01A4BD102ACE01E6BD102ABD08CDCE01A4BD10C0
S1230EE02A4D27E8F6010CBD0A5A5D23DFB7010C39CE0680BD102A8601CE0120BD08A7CEED
S1230F0001A4BD102ABD08BA36BD093CBD1030BD1030BD1030BD10308603B70113A600BDCF
S1230F20093CBD1030087A011326F2BD1030BD1030A600BD102708324C811526BF39CE0120
S1230F409BBD0A464D2303BD0F6FBD0A464D2303BD0FA9BD0A464D2303BD0FC5BD0A464DD7
S1230F602303BD0FD8BD0A464D2303BD100339BD08A7BD09A484034C16B6010D10B7010DC2
S1230F80CE0120A603814227060808080820F4BD08A78601B7010BBD0B8EBD08BA6F03CEC6
S1230FA0035DBD102ABD08BA397D0116270139BD08A77C0111CE044ABD102ACE045FBD101E
S1230FC02ABD08BA39BD08A77C010D77010DCE0499BD102ABD08BA39BD08A7BD0A06B701A5
S1230FE010A6012BF66301BD0A16B60110A100270608A1002701086300CE04B9BD102ABDC4
S123100008BA39BD08A7BD09A484034C16B6010D1BB7010DCE044ABD102ACE046FBD102A23
S11E1020BD08BA397EC0067EC00336BDC0093239368620BD102732397EC000D4
S9030000FC
